:020000040000FA
:0600000000308500072816
:08000800AD0A0B1109000313FE
:10001000831207309900A0308B00003083168C00CB
:10002000C53081000C3085008312203084008001AF
:10003000840A041F17280030AB001D222130D4236E
:10004000AE002430D423B1002230D423B800B30052
:100050000230D423BE001E30D423C0002330D4236A
:10006000AC00AC182C150430B5001930C3003C129C
:100070000610ED213F205C20FD202B223A28203065
:10008000B9001330A900043005052A0603194E28CB
:10009000C320B90B51280430AA063F282A30A900F2
:1000A0004828C320043005052A0603194128C32027
:1000B000DF20A90B512808002508A1002608A2006E
:1000C0002708A3002808A400A501A601A701A801EC
:1000D000253084006E2076207E2008000830A9009C
:1000E000A120A420800DA90B7028C328840AA12078
:1000F000A420800DA120A420800DC328840A0430F0
:10010000A900A120A420800C840AA120A420800C96
:10011000A90303198D2884038128800E8403800E8F
:10012000C328043005052A060319B90A08002A1D48
:100130009D28C320051D99280800C32005199D2866
:1001400008002A199D289928AD01C320043005050F
:100150002A060319AE28AD18BC28A528C320C32041
:10016000C320B9019120C320C3209120C320DF20E8
:1001700091200230390208002030C2002F08C1004F
:10018000BE2397201E282B18D2280512010C7F3978
:100190000319CE282F02031C05100800AF08031D09
:1001A000051408000510010C7F390319DB282F0204
:1001B000031C05120800AF08031D05160800BC1C2F
:1001C000FA2832082F02031CF82803103B0D2C1CC0
:1001D0003B08323E2C180A3EA000010CA002031876
:1001E000C3287D3C031CF6280610C3280614C32828
:1001F0000614C328AC180610C32821082502031DC5
:10020000242922082602031D242923082702031D6E
:10021000242924082802031D24292108031D142948
:100220000130230203197A2A21082E0203191E29FC
:100230002C1F242921083102031D2429C32023084F
:1002400024020319B129252908003C162808FE3E7E
:1002500003194C29FF3E03190513FF3E03198613AA
:10026000FF3E03195229FF3E03199D21FF3E03194A
:100270008221FD3E03195729FF3E03190517FF3E52
:1002800003198617FF3E03194F29FF3E0319A721C3
:10029000FF3E03199021CB292308073C7629230828
:1002A000F83E76292308073C03186A297629083086
:1002B0002702031C762903192429FD3E031905177B
:1002C000FF3E03198617FE3E0319A721FF3E0319BF
:1002D0009021CB2903198221FF3E03199D21FE3E67
:1002E00003198613FF3E03190513CB29240801398E
:1002F0002B060319CB2924080139AB002522013034
:10030000A300CB29AC1E8E29BC1E0800B9002230E8
:10031000D423B800B300BC123908080086100800C6
:10032000AC1E9B29BC1A0800B9000130B800B3000C
:10033000BC1639080800861408002C1DA529AC1C21
:10034000A329BC1008003C110800061008002C1D51
:10035000AF29AC1CAD29BC1408003C1508000614DC
:100360000800C3202308013A031DC6293C18BC29F4
:10037000FF30B4000430B5003C1871223C18CB2982
:100380003C14AB090130AB052522CB29AC18BC14B9
:100390003C1CCB293C10C320ED212308013A031952
:1003A000EA292308BB003C19E2290310BB0DAC1F4E
:1003B000E629A2080319E629221CBB0AA218E6298D
:1003C000BB0AE6293C1EE6293030BB073B08D42394
:1003D000B2000800B201AF0108002C1A0F2A2B1836
:1003E000002A85108516AF0803198512AC1D8516E5
:1003F0003C1A0800A218FE2905130800051708007A
:1004000085128514AF0803198510AC1D85143C1A9C
:100410000800A2180D2A86130800861708002B185A
:10042000172A8510A2188516A21C851208008512AD
:10043000A2188514A21C851008002030D423AF0018
:10044000B2002530D423AB0008002530C2002B08B1
:10045000C100BE2308003808013C031D322A3208BF
:10046000AF00C3283C1232082F020319C328B30B74
:10047000C3283E082F020318462AB2080319432A4C
:100480003E08AF00462AAF01B30AC32832082F0244
:10049000031C4C2AAF034D2AAF0A3808B300AD0144
:1004A0002630D423C3202F08BF00C10B582A5C2A52
:1004B000BF070318AD0A552A0430C100C320AD0C94
:1004C000BF0CAD13C10B5E2AAD080318692AAD0C31
:1004D000BF0C2730D4233F084102031C0030B30770
:1004E000C328B40B0800752A0800FF30B400B50B10
:1004F0000800AE2AC30B0800B22BB600B60A0B30B8
:10050000BC1BDA2BB60B852A080085168514DA2366
:1005100085128510DA23822A0230B6002F30802A15
:100520009B222308013A0319902A9B222308013AAF
:10053000031D952A08003F205C2021082502031D89
:100540009B2A22082602031D9B2A23082702031D3B
:100550009B2A24082802031D9B2A0800BC1009308E
:100560007D2201307D229022E023B9030319DF2A86
:10057000B9030319E72AB9030319F22AB9030319C6
:100580002C2BB9030319422BB9030319542BB903BC
:100590000319562BB9030319582BB90303196B2BF5
:1005A000B90303197D2BB9030319902B0430B90249
:1005B00003199E2B21080319AA2B8C22B32A7D2212
:1005C00090222130C2002108C100BE23B12A7D2221
:1005D00090222230C200E0233908C1002230C2003C
:1005E000BE23B12A7D229022E023C2000310C20D57
:1005F00021080319112B10303902031C012B8C2206
:10060000F32A39087D229022E0230310B90DB91F87
:100610000B2B8C22032B3908C100BE2301307D2215
:10062000F32A0630B600D423B900B6033603D42328
:10063000B9020310390CC1073608C200BE23831665
:100640009C18202B8312B60A1E3036020318B12ADA
:10065000B60AB60A3608132B7D229022E023043016
:100660003902031C352B8C222D2B2330D423E73069
:10067000C105B9033918C115B91841162330C20094
:10068000BE23B12A7D229022E02303303902031CCD
:100690004B2B8C22432B2330D423C112391CC1167F
:1006A0002330C200BE23B12A7D22B12A7D22B12A85
:1006B0007D229022E02305303902031C612B8C221D
:1006C000592B2330D423F830C1053908C104233015
:1006D000C200BE23B12A7D229022E02303303902DA
:1006E000031C742B8C226C2B2330D423C113391C94
:1006F000C1172330C200BE23B12A7D229022E023FD
:1007000004303902031C882B21303902031C8A2B48
:100710008C227E2B2630C2003908C100BE23B12AAC
:100720007D229022E023B908031D982B8C22912B67
:100730002730C2003908C100BE23B12A9022E0232D
:1007400003303902031CA62B8C229E2BBC13391CB0
:10075000BC17B12AFF30B4000430B50001307D224F
:1007600095211E28902290222130C2002108C1002C
:10077000BE231930C30009307D221E28410883168C
:100780009A008312420883169B008B131C129C1143
:100790001C1555309D00AA309D009C141C119C18FE
:1007A000CF2B83128B17080083169B001C141A088A
:1007B00083120800AD01AD02AD08031DDC2B08005B
:1007C000B901A11FE62BB90A211FB90AA11EEC2B02
:1007D0000330B907211EB907A11DF22B0930B90753
:1007E000211DB907A11CF82B1B30B907211CB90723
:0407F00039080800BC
:02400E00C401EB
:104200000000000012000000140015001600180045
:104210001A001C001E0020002200250028002B0090
:104220002E00320036003A003E00430048004E00A7
:1042300054005A00600067006E0075007C000000AA
:1042400000002A000100A0002A00000010001E004B
:10425000000000000000000000000000000000005E
:104260000000000008000A000C000E001000120000
:10427000150018001B001E002100250029002D003C
:10428000FF00FF00FF00FF00FF00FF00FF00FF0036
:10429000FF00FF00FF00FF00FF00FF00FF00FF0026
:1042A000FF00FF00FF00FF00FF00FF00FF00FF0016
:1042B000FF00FF00FF00FF00FF00FF00FF00FF0006
:1042C000FF00FF00FF00FF00FF00FF00FF00FF00F6
:1042D000FF00FF00FF00FF00FF00FF00FF00FF00E6
:1042E000FF00FF00FF00FF00FF00FF00FF00FF00D6
:1042F000FF00FF00FF00FF00FF00FF00FF00FF00C6
:00000001FF
